:030000000219FDE5
:03000B000200AA46
:03002B000201656A
:03005B000202F8A6
:030073000202DEA8
:1000800002030406080C10182030406080040608A3
:100090000C10182030406080A0C000070F1F3F0DDB
:1000A0000D04050D050305030302C2AFC0D0C0E077
:1000B000206217E5256002E473E525F4F58A758B67
:1000C00000D262D0E0D0D0D2AF3285268AC262E5BB
:1000D00026F46035306803207210758B00D0E0D0B4
:1000E000D0C2B1C287C281D2AF32C2B1C287C2818F
:1000F000206E0C206609740AD5E0FDE57E4280750D
:100100008B00D0E0D0D0D2AF32758A00C28DD262DF
:1001100001FF01B9306805206602D2B101B930682B
:1001200005206602D28701B9306805206602D281B7
:1001300001B9C28230680A2066077408D5E0FDD292
:10014000B101B9C28630680A2066077408D5E0FD9F
:10015000D28701B9C28030680A2066077408D5E0EA
:10016000FDD28101B9C2AFC2AD53E6EFC0D0C0E04D
:10017000D2D3D2AFC2CEE52A6007207449152A2116
:10018000C67800790020742EE580307E01F430E5D9
:100190000278FF53DACF207E0343DA20307E034318
:1001A000DA10C2D8C271E580307E01F430E5027900
:1001B000FFC3E89970CB306103752A18207403756A
:1001C0002A18885FD27020740DE52B6004152B214E
:1001D000D643DA01C2D82070024134A85F20610200
:1001E000C2702074367982B70431C3E894F04003BA
:1001F00074F0F8E8C4540F28F87984B70302411B5F
:10020000C313C3138721200802C313200A06C3C8DF
:1002100098F8411B28F8500374FFF88822E52D5404
:10022000066011E533C313C31324062522F52250BB
:10023000037522FF7882B60459852224A824C3E5D9
:100240002495644002A864C3E895664002A86688C5
:1002500025E56970024185C3E8AA699A5003E8FA66
:10026000E4F9EAC333FBE56BF45B29400D256AF83A
:10027000E56A6002156A400B41850AC3E56A9A5037
:1002800002056A78FF8826C26EC3E52694F840020C
:10029000D26EC3E52594404002D26420CF0AD0E05C
:1002A000D0D043E610D2AD32C2CF053A7801E52A6C
:1002B0006005307402152AC3E55F9401400575623C
:1002C0000041D4756300756C00E5622401F562504D
:1002D000037562FFD0E0D0D043E610D2AD32C2AF9A
:1002E000C0D053E67FC260759100855694855795BE
:1002F000759104D0D0D2AF32C2AF53E6EFC2ADC0D9
:10030000D0C0E0C0F0D2D3D2AFA8FBA9FCC2D83095
:100310007102615F53DACF207E0343DA10307E032F
:1003200043DA20D271E580307E01F420E5026136A7
:1003300088278928A18C53DACF207E0343DA203026
:100340007E0343DA10C2D8C271307402A1787800FB
:10035000E580307E01F430E502A178885FA160532A
:10036000DACF207E0343DA20307E0343DA10C271F5
:10037000206102813853DACF207E0343DA10307EC9
:100380000343DA20C2D8D271885A895BC3E89558F2
:10039000F8E99559F97B007E087A00C3E8948CE966
:1003A00094005005755E00812A882178A2E6A82174
:1003B0006055C3E894C8E994005008E4D2E4FB7A9D
:1003C0000A8105C3E89468E994015008E4D2E3FB8C
:1003D0007A0F8105C3E894D0E994025008E4D2E290
:1003E000FB7A1E8105C3E894A0E994055008E4D285
:1003F000E1FB7A3C8105C3E89498E994085008E44D
:10040000D2E0FB7A787E00C3E8955CFCE9955DFD5F
:1004100030E70AECF42401FCEDF43400FD755E00D5
:10042000C3EC9AED9E5003755E01885C895D855A28
:1004300058855B597802A160C3E89527F8E99528AB
:10044000F9307C02A144307B02A144307A02A13D04
:10045000207502815BE9FDE8FC817AE9C313F9E8C4
:1004600013F8307902A13DE9C313F9E813F83078A5
:0F04700002A13DE9C313FDE813FC20612CC3EC8E
:10047F00941CED940240028191ED701EC3EC94C860
:10048F0050180529E52970021529C3E529940A504A
:10049F0002A178755F00D270A178E5296002152955
:1004AF007888E6F97400207F087896B90302789E61
:1004BF00E624FAFEE43400FFC3EC9EFCED9FFD92B0
:1004CF0008B90310A2085007207609D27681E330CD
:1004DF007602C276A2085016B9030DECF42401FC83
:1004EF00EDF43400FD0204FD78007900A144B90356
:1004FF0015EC33FCED33FDC3EC940AFCED9400FDD9
:10050F0050047C007D00C3EC94FFED94004006780E
:10051F00FF7900A144EC8575F0A4C5F0A2F733F87C
:10052F007900400302056078FF7900020560E9C396
:10053F0013F9E813F8307C0EE9600278FFC3E81373
:10054F0038F8E43400F9C3E894FFE99400400278E6
:10055F00FF885FD270206102A178741FF4552F4B72
:10056F00F52FC274EB7002D274752A1830740375AC
:10057F002A0A306102A18C20740353DAFE2074031F
:10058F00752B06D0F0D0E0D0D0D2AD43E610327943
:10059F00010205BC79030205BC790A0205BC791E6C
:1005AF000205BC79640205BC79C80205BC7817E462
:1005BF00D5E0FDD8FAD9F6227A147B780205E37AD2
:1005CF00107B8C0205E37A0D7BB40205E37A0B7B7B
:1005DF00C80205E37902B27DE4C286D5E0FDD28779
:1005EF00D5E0FDC287D5E0FDD286D5E0FDD2B1E5DD
:1005FF0076D5E0FDC2B17496D5E0FDD9D9EAF8D52C
:10060F00E0FDD8FBDBCEC28622C37C007D0075F0F7
:10061F000005F0EA33FAEB33FB50F6EB13FBEA136A
:10062F00FAC3E9FFE8FEE89AF8E99BF95004EFF9FD
:10063F00EEF8B3EC33FCED33FDD5F0DFEDF9ECF86C
:10064F0022E889F08A20D2D4F8A9F07B0030F70B8A
:10065F007BFFF42401F8E9F43400F9E88520F0A4D5
:10066F00ADF0F8E98520F0A4AFF0FEED2EF974009F
:10067F003FFA7C04C3EA13FAE913F9E813F8DCF440
:10068F008BF030F70AE8F42401F8E9F43400F9E8C4
:10069F0089F0C2D4F8A9F0227882B60403020702C7
:1006AF00C3E55F940140030206CC852224E4F5459F
:1006BF00F546F547F548F549C26D0207027882E61F
:1006CF00FCD26DE522F523783879C7AA40AB41C338
:1006DF00EB13FBEA13FAEC146013C3EB13FBEA13EF
:1006EF00FAEC14146007C3EB13FBEA13FAD1188862
:1006FF0045894622C3E5459523F8E5469400F95010
:10070F000CC3E89480E994FF4016020733C3E894C2
:10071F007FE994005003020733787F790002073393
:10072F00788079FF884A894B22E54A2547F8E54BBF
:10073F003548F9854B20E4300701F43549FA30E7A5
:10074F0009C3EA94F04015020771C3EA940F5003EE
:10075F0002077178FF79FF7A0F020771780079002D
:10076F007AF0C3E5249564500AC374019524500BA5
:10077F0002078FE54B20E70E02078FE54B30E706A8
:10078F00884789488A492278A4E6FAC3E54A33F8AC
:10079F00E54B33F9D150E930E70BC3E89480E99486
:1007AF00FF4013E1C9C3E8947FE994005002E1C907
:1007BF00787F7900E1C9788079FFE820E715C3E5F4
:1007CF002398F84009C3E8940140030207F0780129
:1007DF000207F0E8F424012523F840030207F0781C
:1007EF00FF884C2278A5E6FAA848A949D150E930EC
:1007FF00E70CC3E89401E994FF4016020824C3E80C
:10080F0094FFE99400500302082478FF790002084E
:10081F0024780179FFE920E715C3E54C98F84009E2
:10082F00C3E89401400302084B780102084BE8F437
:10083F002401254CF8400302084B78FF88242278C6
:10084F00FFC26420693D206A12D264C3E541940A55
:10085F004009C3E52594405002C26479A1E76023A3
:0D086F00E541601F74FF8541F0848539F07C
:10087C00306A0375F005A4F8C5F0600278FFC3E890
:10088C0095675002A867886622C3E5409440E5410D
:10089C009401E56650031401A6046002F566220279
:1008AC0008AE2275E890227883E6FFE5E820ECF7A5
:1008BC00A8BDA9BE0573C3E57394084052757300B7
:1008CC00E9FA79A0E76044EA7007E574601B020856
:1008DC00E9C3E895746010E5745006600C140208C6
:1008EC00F50460F90208F5E574F574C394A8401B8F
:1008FC007564C0C394054013756480C39405400BA4
:10090C00756440C39405400375640075BB0622E50D
:10091C00642410500274FFF5647982B704022142FA
:10092C00C3A864E524985002A824C3E89566400245
:10093C00A86688258826E573B4070375BB1E227448
:10094C003279A687F0A4C5F0A2F733F8C3E8956412
:10095C004002A86488228824882588268867227506
:10096C0040007541F022C2AF75C820A8CCA9CDAA11
:10097C003A30CF010A75C824D2AFAB3BAC3C883BB4
:10098C00893CC3E89BF8E99C206908F9306702416F
:10099C008721E4AD3D8A3DF9EA9DFA600478FF7940
:1009AC00FFAE3EAF3F8B3E8C3FC3EC9FFCC3E99C3C
:1009BC00F542A83BA93CC3E89EF8E99FF9C3E54181
:1009CC0013FBE54013FAE82AF540E93BF5415006E4
:1009DC007540FF7541FF412EAA40AB41AC40AD4183
:1009EC007E047F02C3EB940440021E1FC3EB9408E9
:1009FC0040021E1FC3ED13FDEC13FCDEF7C3EA9C93
:100A0C00FAEB9DFBEF6009C3E913F9E813F8DFF784
:100A1C00EA28FAEB39FB8A408B4150067BFF8B406E
:100A2C008B41C3EB94025002D2673069047F0341BF
:100A3C00597892E6FFC3E537948240110FC3E5372E
:100A4C0094A040010FC3EF940640027F057E05E59C
:100A5C0041C4540FF9E541C454F0F8E540C4540FB7
:100A6C0028F8C3E89EFAE99400FB4009C3EA940213
:100A7C00EB940050047A02E4FB41D3AA40AB41EB67
:100A8C00C4FEEAC4540F4EFCC3EA9CFAEB9400FB80
:100A9C00C3E813C313F8EA28FAEB3400FB8A408B43
:100AAC0041C3EB94024002C2677805EBC4FE7B00A5
:100ABC00EAC4540F4EFAC3EA98FA4005C3940250A4
:100ACC00027A027892E6FF30600241D38552568555
:100ADC005357D26043E680C3E49AF8E49BF930673D
:100AEC0002616DE8FAE9FBD3E913FDE813FC8852C7
:100AFC008953C3EF94036038EF20E00DE82CF8E93C
:100B0C003DF9ECFAEDFB020B28E828F8E939F9C3BA
:100B1C00E82402F8E93400F97AFE7BFFC3EF940372
:100B2C00400E8A548B55884E894F8C508D5161A143
:100B3C00885489558A4E8B4F8C508D51306920C307
:100B4C00E53394034019E542A2E713F8E555F42484
:100B5C000138400B20E7087554FFF42401F555616A
:100B6C00A1E8FAD3E813FC8852C3EF94036020EF9A
:100B7C0020E007E82CF8ECFA618DE8282402F87ADA
:100B8C00FEC3EF940340088A54884E8C5061A188B0
:100B9C00548A4E8C50E56BC3335002646BF56B304A
:100BAC00600261AB753402D26043E680E52D5406D9
:100BBC006026A840A941C3E913F9E813F8C2AF5362
:100BCC00E67F759100C3E498F594E499F5957591D9
:100BDC0004D26043E680D2AF22D265754400752002
:100BEC0000306B03752040020C04D265754400750F
:100BFC002040306B03752000D2AF7801206722E5CE
:100C0C002D54066002C265C3E54194054013780279
:100C1C009405400878039405400278063069027800
:100C2C000A206019E544601530690AC3E533940362
:100C3C004003D53406D2AFD26C81D571B3D2AF009C
:100C4C0000C2AF206726E541C3FB940F40027B0F27
:100C5C00EB240530730123306A02742820620123CF
:0E0C6C00F93069027982E58BC39940B50544E1
:100C7A00E59B5440B5200281BF30690A08C3E89455
:100C8A000A400108812D2065028104C26553E67F6E
:100C9A007591003067107594007595FE759104D2B0
:100CAA006043E6808104AE40AF41C3E49EF594E41C
:100CBA009FF59581A6C3E5339402500281043065FD
:100CCA00028104D80281D3812DC26C53E67F7591CB
:100CDA0000855494855595759104854E56854F57D0
:100CEA00D26043E680D2AFE52D54066008206A023E
:100CFA000533020D0F306C0D206B0A206507158134
:100D0A00158102158C22780030640530650278015D
:100D1A00E53775F007A4F9E5F028F5F0E9A2F01334
:100D2A00A2F113A2F213F537C394785003753778FA
:100D3A00C3E53795384008D266C2B1C287C281304E
:100D4A006002A149855056855157D26043E68022F8
:100D5A00207D11C2AF754302C286D282D2AF759F7F
:100D6A0002020F29C2AF754302C286D280D2AF7582
:100D7A009F02020F29307243207D20C2AF754303C0
:100D8A00900143757E40C281C280306204D287A13D
:100D9A009DD286D2AF759F03020F29C2AF75430356
:100DAA00900143757E40C2B1C282306204D287A1EB
:100DBA00BDD286D2AF759F01020F29207D17C2AF1F
:100DCA0075430390011EC281306202D287D2AF7589
:100DDA009F03020F29C2AF75430390011EC2B130AF
:100DEA006202D287D2AF759F01020F29207D11C2FC
:100DFA00AF754304C282D280D2AF759F01020F2918
:100E0A00C2AF754304C280D282D2AF759F03020F6C
:100E1A0029307243207D20C2AF7543059001327597
:100E2A007E04C287C286306204D2B1C139D282D26C
:100E3A00AF759F02020F29C2AF7543059001547521
:100E4A007E01C287C286306204D281C159D280D261
:100E5A00AF759F02020F29207D17C2AF7543059017
:100E6A000114C287306202D2B1D2AF759F02020F5B
:100E7A0029C2AF754305900128C2873062EBD2813F
:100E8A00D2AF759F02020F29207D11C2AF754306AA
:100E9A00C280D286D2AF759F03020F29C2AF7543B3
:100EAA0006C282D286D2AF759F01020F29307242E2
:100EBA00207D20C2AF754301900154757E01C2B1F5
:100ECA00C282306204D281C1D5D280D2AF759F016D
:100EDA00020F29C2AF754301900132757E04C281A7
:100EEA00C280306204D2B1C1F5D282D2AF759F03FB
:100EFA00E129207D16C2AF754301900128C2B130A5
:100F0A006202D281D2AF759F01E129C2AF75430156
:100F1A00900114C281306202D2B1D2AF759F03C26E
:100F2A006622900112757E00C2B1C287C281C28256
:100F3A00C286C280C262227880760908760908765B
:100F4A00040876FF0876030876FF08760908760310
:100F5A00087601087601788C76010876FF0876FF14
:100F6A000876FF0876FF0876FF0876030876FF08FA
:100F7A0076FF0876FF0876250876D0087628087660
:100F8A00500876040876FF08760208760008767A12
:100F9A000876FF08760108760108760008760322AB
:100FAA007887E6FFC272BF0302D2727888E6C394DA
:100FBA00036008C27DE630E102D27DC27E7889E60E
:100FCA0030E102D27EC3EF94026008758E01D273BB
:100FDA00020FE2758E00C273227880E614900080B8
:100FEA009378A4F67881E6149000809378A5F67831
:100FFA0086E61490008D9378A6F6789CE67538FFFD
:10100A0075390CB402067538A075390AB403067529
:10101A00388275390578A3E61490009A93F5691217
:10102A000F2C22227896E6FA7897E6FB7888E6B4BF
:10103A000305C3EB940EFB307F047A007BFFC3EBFE
:10104A009AFCC3948250027C827575000575EC8502
:10105A0075F0A4C3E5F0947D40F222D27F112E12DE
:0F106A0005AD7A007B007C101205A3E55F2AFA22
:1010790074003BFBDCF37C04C3EB13FBEA13FADCDF
:10108900F7FEC27F112E22E5EF20E6037520000549
:1010990020903DFFE520146006901FFF1460009327
:1010A90004600375EF1253D9BF7581C043FF8012E5
:1010B900059E75EF0243B203E5B3240420E70DF55D
:1010C90021E5B120E0068521B343B101120F2C754A
:1010D900803875A4C775F1FF75D4DF7590FF75A5C4
:1010E9000075F20075D50075A0FF75A60075F300AF
:1010F90075D60075B0E475A71B75F4FF75E241E478
:10110900F8F6D8FD756B01120F411215CE78988645
:1011190076753001C2AF1205B71205C71205AD12B7
:1011290005CE1205AD1205D51205ADC2AF78FA7913
:10113900FA308507D9FBD8F7021C00120FAA120F43
:10114900E3112D112E78988676120F2C758850751B
:10115900891275C82475910475D84075A82275B887
:101169000275E690759B80759D0075D10E75BC580A
:1011790075BB0675BA1F75E88012059ED2AF1208B5
:10118900AB53DACF207E0343DA20307E0343DA10F3
:1011990043DA01C2D8C2711205B7D2617B037A0C56
:1011A900E55E70077A0CDB030211341205AD20707D
:1011B90003021134C270E55FC3940240E1E52F5484
:1011C9001F856160F561B560D5DAD5C26153DACFA3
:1011D900207E0343DA20307E0343DA10C2D8C2717D
:1011E90078A2E67008D274E52F54E0F52FC2757520
:1011F90029001205B2307409C3E529940A4002D2C4
:10120900751205A378023074027800C3E55F98402F
:10121900F0C2AF1205C71205C71205C7D2AF120532
:10122900B7754D007888E6B40302610B1205A378FF
:101239008CE6C39401500302130BE530C3940150AB
:101249000302130B207435C3E55F94FF50030213A7
:101259000BC2AF1205DCD2AF1205B2C3E55F940130
:1012690050EFC2AF1205C71205A81205C7D2AF12B7
:1012790005B2C3E55F94FF40E90217767F02D27F8A
:10128900112E1205B2C2AFC27F112EAE5FC3E55F48
:10129900947FD2AF407612059EC2AF1205DCD2AF61
:1012A900DFDC1165C3EE94057897F61205B71216BF
:1012B900101216F97F0AD27F112E1205B2C2AFC2DF
:1012C9007F112EAE5FC3E55F947FD2AF50E6120562
:1012D9009EC2AF1205C71205A81205C7D2AFDFD645
:1012E9001165EE24057896F61205B7121610121735
:1012F900281205B2112EC3E55F94FF5002414D0239
:101309001776C3E55F954D4003855F4D1205B278A9
:10131900017988E7B403027805C3E55F9840024183
:101329002DC2AF1205DC1205DC1205DCD2AF1205A5
:10133900B7753000E4F531F5320531E531F470392E
:101349000532789AE67819146012783214600D78AB
:101359007D14600878FA146003753200C3E5329889
:10136900401715327531B478998676C2AF1205DC0B
:10137900D2AF789886761205B21205A8E52A7005CB
:10138900307402213478012074027806C3E55F982D
:1013990040A77888E6C3940360031205B2E52A7072
:1013A90003021134C2AF120F2CE4F522F523F52400
:1013B900F525F526F56AD2AF7885E6C333F568E4F5
:1013C900F545F546F547F548F549F573F52CF52D3D
:1013D900F53775730875BB1E12059E1208AFE5E84F
:1013E90020ECFBA8BDA9BEE97001F888741208B306
:1013F90075730875BB1E7887E6FE7602120FAA7808
:1014090087EEF6C2AF7564FF12094B852264852207
:1014190065852266D2AF752201752401752501758E
:10142900260185636C756D017888E6B40307C27D72
:10143900307602D27DD268D269753300120E9212CB
:101449000EB712096B12097212096B12097212098D
:101459006B02146AC2AF120FAAD2AF75730075BBC3
:0D14690006120BF61206A7120D10120D5AF6
:10147600120972120BE5306D03120703206703127F
:10148600084E306703120895120D10120D7F1209CF
:1014960072120BF6306D03120738120D10120DF68C
:1014A600120972120BE5306D03120796120D101217
:1014B6000E1B120972120BF6306D031207F3120D92
:1014C60010120E921209721208AF120BE5120D10CD
:1014D600120EB71208B3120972306935206B3285C5
:1014E600676485676585636C756D0179187A0CC3C9
:1014F600E53399400FC269D26A8A35856764856784
:1015060066021517C3E55F9401400302146A0215CB
:1015160094306A1B206B18E535147004C26A815D2D
:10152600F535C3E55F9401400302146A021594750C
:101536003600C3E56278FA985054307404E52A60A0
:101546004D7888E6B40317207D05207607A1643020
:101556007602A164206B07D26B85676481A978F057
:10156600306B058567647820C3E541985002816A2F
:10157600306B1BC26BC27D307602D27DD26A753566
:1015860012856764816A0536E55F6002A197753644
:1015960000C2AF120F2C7887E6FE7602120FAA78E9
:1015A60087EEF6E4F522F523F524F525F526F5680C
:1015B600C268D2AF12059E120F2C307409C3E536ED
:1015C600940540022134613D901A0D78201216527E
:1015D600E520B4550CA3121652E520B4AA03021551
:1015E600F0120F4112161002160F901A0378807B24
:1015F6000A121652A308DBF9901A0F788C7B181280
:101606001652A308DBF9901A2722C2AF12169112BE
:10161600166B901A00740E121657A37404121657FE
:10162600A37414121657901A0378807B0A12165662
:10163600A308DBF9901A0F788C7B18121656A308AC
:10164600DBF91216A4121682901A2722E493F622C8
:10165600E6438F01538FFD75EF0275B7A575B7F198
:10166600F0538FFE22438F02438F0175EF0275B749
:10167600A575B7F1901A0DF0538FFC22901A0D74D0
:1016860055D157901A0E74AAD157227A3079D0784C
:1016960020901A40D152E520F709A3DAF7227A30D2
:1016A60079D0901A40E7D15709A3DAF922AB77A887
:1016B60078BB01027980BB02027981BB0302798281
:1016C600BB04027984BB05027986BB06027992BB0C
:1016D60007027987BB080279A3BB0902799CBB0A7A
:1016E600027988BB0B027989E8F7227C051205B7D7
:1016F600DCFB22C2AF1205C71205CE1205D51205B4
:10170600DC1205A81205C71205CE1205D51205DC96
:101716001205A81205C71205CE1205D51205DCD290
:10172600AF22C2AF1205DC1205D51205CE1205C7CF
:101736001205A81205DC1205D51205CE1205C71230
:1017460005A81205DC1205D51205CE1205C7D2AFC3
:1017560022AE77AF78C2AF1205C71205C71205C70A
:101766001205A8DEF21205DC1205A8DFF8D2AF22B8
:10177600D1F9D1F1D1F1757701757801757900F15B
:10178600577C05AD5F1205B7C3ED955F70F5C3E5F0
:101796005F9401400AC3E55F94FF40320217B2D15D
:1017A600B3D110D1F9C2AF75EF12D1F1DCD50579FD
:1017B600C3E5799403500280C6D1F10578E5771424
:1017C60090009F93F808C3E57898500280AED1F157
:1017D600D1F10577C3E577940C5002809C120F4136
:0917E600D110C2AF75EF12D1F170
:0319FD0002109045
:101A00000E0414090904FF03FF0903010155AA018B
:101A1000FFFFFFFFFF03FFFFFF25D0285004FF0259
:081A2000007AFF01010003FF41
:101A4000235475726E696779343041232020202039
:101A500023424C48454C4923463331302320202033
:101A60002020202020202020202020202020202076
:101C0000C2AFC2D353D9BF7581C043B20343FF8073
:101C1000752438752503B1C975EF0275E24043F1AB
:101C20002053A4DF75D400D2857DFA780379E67C51
:101C300010752200752300901DD67B0675249875BB
:101C400025013085028142208508D8FBD9F9DCF7CF
:101C500081B4308508D8FBD9F9DCF781B4B189E4C7
:101C600093A3C39A6004DDC381B4DBDBB17B600264
:101C7000812B7B08E493FAA3B15CDBF87A30B15C8A
:101C8000752200752300B17BEAFCEBFDC3ED94FEE9
:101C9000400EB17B8A278B28ED30E0048A828B834B
:101CA000B17B7AC270D8C3ED94FE601350CEBD00F4
:101CB00025EC60097520007521FF0200008100A855
:101CC00027A9280809D804D90281D3B17FEA89AAB3
:101CD000F281C50D81A0C3ED94035049EDA2E092BD
:101CE000007AC5C3E5829400E583941C50902000DF
:101CF00010438F02438F0175B7A575B7F1F030001F
:101D00001FA827A9280809438F01538FFDD804D99C
:101D100002A12089AAE275B7A575B7F1F0A3A10DBC
:101D2000538FFC817C7AC1BD030CE493A3FAB140CC
:101D3000DCF8B138817C817EAA22AB23B15CEBFA5E
:101D4000EA6222752608C3E52313F523E52213F57D
:101D50002250066323A0632201D526EAB1C9B1C986
:101D600075260AEAF4200102D285300102C285B14B
:101D7000C9C3134002C201D526EB22B17FEAFB2082
:101D80008502A17F308502A184752608AE24AF2587
:101D9000C3EF13FFEE13FEB1CDB1C9C3EA13308513
:101DA000024480FA30E703632201C3E52313F523DD
:101DB000E52213F52250066323A0632201D526D91C
:101DC000E52265236523F52222AE24AF250E0FDE22
:101DD000FEDFFCD20122424C48656C693437316326
:041DE000F3100601F5
:00000001FF
